:10000000830100308A000428203084003A300D201B
:100010008301842904068001840A0406031900343C
:020020000A28AC
:1000620083123808BB003708BA00B81F0800BA0963
:10007200BB09BA0A0319BB0A080090018E018F015D
:100082000C1010148312851A48280C1C4428851E53
:100092004C280C1C482810100C1C0034851E0134FE
:1000A2000234BE01BF010310BD0CBC0C031C60284E
:1000B2003A08BE073B0803183B0ABF070310BA0DF4
:1000C200BB0D3C083D0403190034542883169B00E1
:1000D2001C148312B700370A83169B001C141A08DB
:1000E200BD00BC011A08BA00BB013C08BA070318DC
:1000F200BB0A3D08BB0783120800B9003903031984
:1001020086283908023A031DAA2883129001FF307B
:10011200BA00BB0037083A02B7003808031C380A95
:100122003B02B8008F0037088E000C103903031D04
:10013200A028051510140C1C9C280511A9283908A3
:10014200023A031DA928051610140C1CA628051234
:10015200101083120800B70001303702031CB528C3
:1001620003303702031CB828BA01BB01DC28831212
:1001720090018E018F013703031DC528851DBF28FD
:1001820010148519C228CE283708023A031DCF2839
:10019200851EC9281014851ACC2810100F08BD001E
:1001A200BC010E08BA00BB013C08BA070318BB0A1F
:1001B2003D08BB0708008312080090018E018F01E1
:1001C2008312851DE2281014851EE5280F08AB0056
:1001D2000E08AA008E018F01851DED280F08AD00C3
:1001E2000E08AC0010102B08AA00AB012D08AC00C1
:1001F200AD0100302B02203003192A0203180D2909
:1002020000302D02213003192C02031C0D29A001FC
:10021200A00A0230A100080002308312A000A1014E
:10022200A10A0800B90083169C18152983123908FF
:1002320083169B008312380837040030031D0130F7
:1002420083169A0003108B1B03148B1383161C1541
:1002520055309D00AA309D009C141C1103188B1769
:100262009C1831298312390A83169B00831238089D
:1002720083169A0003108B1B03148B1383161C1511
:1002820055309D00AA309D009C141C1103188B1739
:100292008312080090015B29BF30AA07031CAB033D
:1002A2000C108E0102308F0017308E0010140C1CBF
:1002B20058291010003083122B02423003192A02EF
:1002C20003184D29E830BC000330BD002B08BB00E9
:1002D2002A08BA005220FF30BA00BB003E08BA0218
:1002E200031CBB033F08BB023A08AA003B08AB0051
:1002F2000C108E018F002A088E00101483120C1C21
:1003020080291010080057308316810011309500A3
:100312008312FF23831690000730831299008316FD
:100322009F01093085000030831267203A08AC0033
:100332003B08AD00023067203A08AA003B08AB0038
:10034200DC30B0000530B1000518752AE830AC0089
:100352000330AD00D030AA000730AB008514B601DF
:10036200B60AB401B5018312B6080319762A013020
:10037200AC203A08AE003B08AF00803ABA008530A4
:100382003A02143003192E020318E8293108803A80
:10039200BA0083303A02E93003193002031CDF2924
:1003A2003108803ABA0087303A02D030031930025D
:1003B2000318DF29E830B0000330B1008312B0081F
:1003C2000319B103B003B401B5018514682A83127D
:1003D2002F08803ABA0086303A02A53003192E025D
:1003E200031C0F2A3108803ABA0083303A02E930FE
:0E03F20003193002031C0B2A3108803ABA00AE
:1004000087303A02D0300319300203180B2AD0305B
:10041000B0000730B100B00A0319B10AE429B40AE8
:100420000319B50A3408FA3A3504031D392A851030
:100430003108803ABA0083303A02E83003193002BA
:100440000318262A3008AC003108AD003108803A84
:10045000BA0087303A02D13003193002031C342A23
:100460003008AA003108AB00DC30B0000530B10024
:10047000682A3508803ABA0081303A025F300319A1
:100480003402031C682A3508BB003408BA003B0D4F
:10049000BB0CBA0C3B0DBB0CBA0C3A0C031C522A19
:1004A0008514532A85103508023A5830031934064A
:1004B000031D682AB6012C08B7002D08B8000030CB
:1004C00013212A08B7002B08B80002301321831229
:1004D0003008B7003108B80001307E203008B7007E
:1004E0003108B80002307E20B42983128510B20191
:1004F000B30101308312AC203A08AE003B08AF00D4
:10050000803ABA0083303A02E83003192E02031809
:100510008D2AE830AE000330AF0083122F08803AF6
:10052000BA0087303A02D13003192E02031C9C2AEC
:10053000D030AE000730AF002F08BB002E08BA0045
:100540001830BA070318BB0AFC30BB073A08BE00D4
:100550003B08BF000030BF1BFF30C000C1002D08AA
:10056000BB002C08BA002A08BA02031CBB032B08E4
:10057000BB023A083B080030BB1BFF30BC00BD008B
:10058000C2231830BE00FC30BF00FF30C000C100E5
:1005900020232C083A07B0002D0803182D0A3B072A
:1005A000B10030083202B7003108031C310A3302AF
:1005B000B800831231203B08803ABC0080303C02F6
:1005C000023003193A02031C042B3008B70031082B
:1005D000B80001307E202D08BB002C08BA002A0884
:1005E000BA070318BB0A2B08BB0730083A02B7004A
:1005F0003108031C310A3B02B80002307E2030086B
:10060000B2003108B300792A83123208B7003308E8
:10061000B80001307E202D08BB002C08BA002A0843
:10062000BA070318BB0A2B08BB0732083A02B70007
:100630003308031C330A3B02B80002307E20792ABB
:1006400084018312C601BD1F342B0310FF30BA078B
:10065000BA09031CBB07BB09031CBC07BC09031C6C
:10066000BD07BD094617C61741088039C606C11F18
:100670004A2B0310FF30BE07BE09031CBF07BF098A
:10068000031CC007C009031CC107C1094A2B840110
:100690008312C601C201C301C401C5013E083F0463
:1006A000400441040319572BC030C605622BBA0120
:1006B000BB01BC01BD01F02B0310BE0DBF0DC00D71
:1006C000C10DC60AC11F5C2BC60A0310C20DC30DA3
:1006D000C40DC50D41083D02031D782B40083C02A6
:1006E000031D782B3F083B02031D782B3E083A027E
:1006F000031C8A2B42143E08BA023F08031C3F0F1A
:10070000BB024008031C400FBC024108031C410F00
:10071000BD020310C10CC00CBF0CBE0CC6034608C2
:100720003F39031D652B461FA22B0310FF30BA076C
:10073000BA09031CBB07BB09031CBC07BC09031C8B
:10074000BD07BD093A08BE003B08BF003C08C00019
:100750003D08C1004208BA004308BB004408BC0081
:100760004508BD00C61FF02B0310FF30BA07BA09B9
:10077000031CBB07BB09031CBC07BC09031CBD074A
:10078000BD09F02B84013A08C2003B08C3003C08B5
:10079000C4003D08C500BC01BD01BA01BB01031086
:1007A000C50CC40CC30CC20C031CE42B3E08BA07D6
:1007B0003F0803183F0FBB0740080318400FBC0752
:1007C00041080318410FBD0742084304440445048F
:1007D0000319F02B0310BE0DBF0DC00DC10DCF2BA3
:1007E0008408031900343D08800084033C0880001D
:0E07F00084033B08800084033A088000003434
:02400E00C43FAD
:10420000E8000300D00007000000000000000000EC
:00000001FF
